:020000040000FA
:100000000313831207309F0000308B0000308500FF
:10001000003086008316C53081001E308500F03028
:1000200086008312A601A001AA0103102A14A501CB
:1000300006148615061A2514861AA514061B2515FE
:10004000861BA5150610861173209620F7203820F0
:100050003120382031203820312038203120312003
:1000600024285F30A30000000000A30B3328080001
:1000700003308A00200800238A01A7000830A4006A
:100080000510A70D6D20031C0514672005146D20B5
:10009000A40B402805106D20A61E0514672005142A
:1000A0006D2005106D20A61E0514672005146D2017
:1000B0002108A7000830A4000510A70D6D20031C1F
:1000C0000514672005146D20A40B5C280800083077
:1000D000A3000000A30B692808000230A300000061
:1000E000A30B6F280800A8010430A900860103149F
:1000F000860D0310061A9428A80A861A9428A80ABE
:10010000061B9428A80A861B9428A80A85189428F8
:10011000A80A05199428A80A85199428A80A051A76
:100120009428A80AA90B782886010800AA1EE828A6
:10013000A81AF028AA0103102A1404302802031870
:10014000A4280130FA20E228083028020318AD283C
:100150000230FA200430A802E2280C3028020318EA
:10016000B6280130FA200430A802E2281030280214
:100170000318BF280230FA200830A802E228143001
:1001800028020318C8280330FA201030A802E228F9
:10019000183028020318D1280430FA201430A8029D
:1001A000E2281C3028020318DA280330FA20143021
:1001B000A802E228203028020318E2280430FA209E
:1001C0001830A80202308A00280800228A01A10003
:1001D0002A18F328AA18F3282110A110AA0D080044
:1001E000A101A00108002114A114AA0D0800851C7A
:1001F000F72808009B0083161C1483121A08A0001D
:060200002508A00708001C
:10040000820700340C3430343C34C034CC34F03403
:04041000FC34003484
:100600008207AA34C03480343034F034B03420341B
:10061000E034A0340C34CC348C343C34FC34BC3462
:100620002C34EC34AC340834C83488343834F834DE
:10063000B8342834E834A8340334C334833433342E
:10064000F334B3342334E334A3340F34CF348F344E
:100650003F34FF34BF342F34EF34AF340B34CB345A
:100660008B343B34FB34BB342B34EB34AB340234AB
:10067000C23482343234F234B2342234E234A2341A
:100680000E34CE348E343E34FE34BE342E34EE344A
:10069000AE340A34CA348A343A34FA34BA342A3496
:1006A000EA34003440346034973470344834683469
:1006B0005834783444346434543474344C346C34A2
:1006C0005C347C3442346234523472344A346A3496
:1006D0005A347A3446346634563476344E346E3472
:0206E0005E3486
:02400E00293F48
:104200000200140028003C00000000000000000034
:10421000000000000000000000000000000000009E
:10422000000000000000000000000000000000008E
:10423000000000000000000000000000000000007E
:10424000000000000000000000000000000000006E
:10425000000000000000000000000000000000005E
:10426000000000000000000000000000000000004E
:10427000000000000000000000000000000000003E
:00000001FF
